:020000040000FA
:0600000050EF08F01200B1
:0600080004EF10F01200ED
:060018000CEF10F01200D5
:02002A000000D4
:04002C00550EA76E58
:10003000AA0EA76EA68212000001420E6D6F020E7C
:100040006E6F010E6F6F12000001606B6951605D91
:100050001EE260C000F0016A026A6A510024F36E79
:100060006B510120F46E6C510220F86EF4CFF7FF53
:10007000F3CFF6FF0800F5CF61F06051EA6A6D0F2B
:10008000E96E000EEA2261C0EFFF602BDFD7F86A4D
:1000900012000001000E6A5D200E6B59000E6C59B3
:1000A00008E3D880FF0E6A555F0E6B55000E6C5545
:1000B00001E239D0606B6951605D34E260C000F0EC
:1000C000016A026A6A510024F36E6B510120F46EDA
:1000D0006C510220F86EF4CFF7FFF3CFF6FF080063
:1000E000F5CF61F06351641165111AE16051EA6A5C
:1000F0006D0FE96E000EEA22EF50615D11E060C005
:1001000000F0016A026A6A0EE96E000EEA6EEE50B5
:100110000024636FEE500120646FEE500220656F83
:10012000602BC9D7F86A120063C000F064C001F008
:1001300065C002F0036A005000016D6F63C000F0FB
:1001400064C001F065C002F0036A080ED890033263
:10015000023201320032E806F9E1005000016E6F10
:1001600063C000F064C001F065C002F0036A100EC5
:10017000D8900332023201320032E806F9E1005031
:1001800000016F6F1200840EA66E0001000E6A5D02
:10019000200E6B59000E6C5908E3D880FF0E6A558B
:1001A0005F0E6B55000E6C5501E22ED0606B6951ED
:1001B000605D27E26051EA6A6D0FE96E000EEA2287
:1001C000EFCF03F060C000F0016A026A6A510024B8
:1001D000F36E6B510120F46E6C510220F86EF4CF77
:1001E000F7FFF3CFF6FF03C0F5FF0C001F0E6015FD
:1001F0001F0803E06905605D01E118DF0001602B65
:10020000D6D7636B646B656B12000001000E6A5DEC
:10021000200E6B59000E6C5908E3D880FF0E6A550A
:100220005F0E6B55000E6C5501E225D0606B695175
:10023000605D20E2940EA66E6051006E016A060EAB
:10024000D89000360136E804FBE1026A01BE02687C
:1002500000016A510024F36E6B510120F46E6C5161
:100260000220F86EF4CFF7FFF3CFF6FFDFDE0001D8
:10027000602BDDD7F86A1200A66A0001606B695135
:10028000605D0EE26A516025A96EA6806051EA6A3F
:100290006D0FE96E000EEA22A8CFEFFF602BEFD7BB
:1002A00012000001606B6951605D13E26A516025C4
:1002B000A96E6051EA6A6D0FE96E000EEA22EF50F6
:1002C000A86E040EA66EB2DEA6B2FED70001602BA9
:1002D000EAD71200C40EA66E0001606B6951605D22
:1002E00020E26051EA6A6D0FE96E000EEA22EFCF5C
:1002F00003F060C000F0016A026A6A510024F36EE4
:100300006B510120F46E6C510220F86EF4CFF7FFB0
:10031000F3CFF6FF03C0F5FF0C0088DE0001602B71
:10032000DDD7F86A1200400EE66E680EE66E000E2B
:10033000E66EF5EC05F0E552E552E552000801E302
:1003400089D00001606B00016851FF0A70E0FA0A71
:1003500069E0010A54E0070A4DE00A0A38E0010AA0
:1003600034E00A0A2DE0030A18E0070A16E0700AD2
:1003700001E06FD061DE0001040E606F04010CBF6C
:10038000FDD7400EE66E680EE66E000EE66EBBEC24
:1003900005F0E552E552E5525DD056DE050E00014E
:1003A000602704010CBFFDD7400EE66E680EE66EB6
:1003B000000EE66EBBEC05F0E552E552E5524AD080
:1003C000E2DE0001010E606F45D063DE43D0ACDE9B
:1003D000050E0001602704010CBFFDD7400EE66E3C
:1003E000680EE66E000EE66EBBEC05F0E552E552D7
:1003F000E55230D00ADF0001010E606F2BD03CDFE8
:10040000050E0001602704010CBFFDD7400EE66E0B
:10041000680EE66E000EE66EBBEC05F0E552E552A6
:10042000E55218D03EDF0001010E606F13D052EC90
:1004300006F00001666B676B00016607000E675BE4
:1004400000016651671103E000000000F5D7FF00CE
:0604500001D000D01200F3
:0A04560004011051600BE842E84277
:10046000E842E842E842000901E055D01151070A8C
:1004700051E00B0A4FE0070A40E0010A2CE00B0AAA
:1004800028E0020A26E0030A22E0080A12E0010A34
:100490000EE00F0A0AE0030A01E03CD00001010E61
:1004A000B36F0001040EBA6F36D036D834D090D86E
:1004B00032D00001010EB36F0001BC0EB46F000E0C
:1004C000B56F0001BB930001010EB86F24D0A8D80E
:1004D00022D0F5D820D00001010EB36F04011451D1
:1004E0000001B46FB56BBD0EB427000EB52300013B
:1004F000BB930001010EB86F0ED00001010EB36F67
:1005000004011451EA6ABD0FE96E000EEA2212C41A
:10051000EFFF01D000D01200800E0401105D57E102
:100520001351030A34E0010A10E0030A01E04DD040
:100530000001010EB36F0001DE0EB46F0D0EB56F3A
:10054000120E0001B86FB96B40D00001010EB36FFD
:1005500004011251F66EF76AD890F636F736FE0EA1
:10056000F6260E0EF7220900F5CFB4F00A00F5CFFB
:10057000B5F0020E0001F76AB425F66EB551F72208
:100580000900F5CFB8F00A00F5CFB9F01ED0000190
:10059000010EB36F04011251F66EF76AD890F63669
:1005A000F736020EF6260F0EF7220900F5CFB4F04B
:1005B0000A00F5CFB5F0B4C0F6FFB5C0F7FF0800EC
:1005C000F5500001B86FB96B00D00001BB83120079
:1005D0000001010EB36F0F0EE66E710EE66E0F0E88
:1005E000E66EDAEC06F0E552E552E552010EE66EF3
:1005F000BD0EE66E000EE66EDAEC06F0E552E55250
:10060000E55212C4BCF00401125104E10001050ED0
:10061000BA6F05D00001060EBA6FA6EC05F0120005
:100620000401186B196B040110511F0B020A15E02D
:10063000030A0FE0010A01E034D00001010EB36F9C
:1006400002D0040118810001BBA102D0040118836B
:1006500028D00001010EB36F24D00001010EB36F4A
:10066000040114510F0B080DF350016A000F006EC6
:10067000040E01221451800B01E0010E040DF35011
:1006800000010024B66F000E0120B76FB6C0E9FF6D
:10069000B7C0EAFFEF50040B03E00401010E186F2E
:1006A00000D00001B3050AE10001180EB46F040E7A
:1006B000B56F0001BB930001020EB86F1200040178
:1006C000120510E110511F0B00090CE10001010E91
:1006D000B36F030E0401115D03E10001BB8102D081
:1006E0000001BB91040112513AE110511F0B0208A5
:1006F00036E114510F0B000932E00001010EB36F17
:10070000040114510F0B080DF350016A000F006E25
:10071000040E01221451800B01E0010E040DF35070
:1007200000010024B66F000E0120B76F030E040114
:10073000115D07E1840EB6C0E9FFB7C0EAFFEF6EB6
:100740000ED014AF06D0B6C0E9FFB7C0EAFFEF6A1B
:1007500006D0880EB6C0E9FFB7C0EAFFEF6E120000
:100760006C500BE1040100513C0BE842E8420D08DB
:1007700002E108D801D03CD804D0040E6C5C01E141
:1007800047D81200D9CFE6FFE1CFD9FFE6520001EA
:10079000B26BB36BB86BB96B2BEC02F0DF6ADF5056
:1007A000006E016A010E005C000E01581BE20001A0
:1007B000B35101E017D0F76ADF34FE0BF736F66E5F
:1007C0000C0EF6260F0EF7220900F5CF00F00800F8
:1007D000F5CF01F004D001C0FAFF0050F96EFBDF45
:1007E000DF2ADDD7DDD8E552E552E7CFD9FF120089
:1007F000020E0001B25D0AE196D8040100BD03D0EB
:10080000C80E006F02D0880E006F01D00FD9120001
:10081000040E0001BA5D0AE112C46EFF6E500008BA
:1008200003E2050EBA6F02D0030EBA6F0001B205E3
:100830000AE10BD8040104BD03D0C80E046F02D036
:10084000880E046F01D0F2D81200D9CFE6FFE1CFB5
:10085000D9FF020EE1260001080EB85D000EB9595D
:1008600005E2B8C0DEFFB9C0DDFF03D0080EDE6EC2
:10087000DD6A040104930491010EDB500413DFCF01
:1008800005F4000EDB500001B85F010EDB50B95BD0
:10089000180EB66F040EB76F0001BBA31ED0D9CFE0
:1008A000E9FFDACFEAFFEE50ED1016E0B4C0F6FF34
:1008B000B5C0F7FF0800F550B6C0E9FFB7C0EAFFC2
:1008C000EF6E0001B62B000EB723B42BB523DF0665
:1008D000010E01E2DB06E3D71CD0D9CFE9FFDACF66
:1008E000EAFFEE50ED1015E0B4C0E9FFB5C0EAFF35
:1008F000EF50B6C0E9FFB7C0EAFFEF6E0001B62BBC
:10090000000EB723B42BB523DF06010E01E2DB0690
:10091000E4D7020EE15C02E2E16AE552E16EE552E3
:10092000E7CFD9FF1200D9CFE6FFE1CFD9FF020E02
:10093000E126030E04010015E76E010EE7CFDBFF91
:1009400001C4DFFFDE500001B827DD50B923180EC7
:10095000B46F040EB56FD9CFE9FFDACFEAFFEE50DE
:10096000ED1014E0B4C0E9FFB5C0EAFFEF50B6C027
:10097000E9FFB7C0EAFFEF6EB62B000EB723B42B2A
:10098000B523DF06010E01E2DB06E5D7020EE15CCE
:1009900002E2E16AE552E16EE552E7CFD9FF1200CB
:1009A0006D980001B3510CE10401080E016F100EA7
:1009B000026F040E036F840E006F0401046F35D0C4
:1009C000040110AF22D00001B8510401165D0001EE
:1009D000B9510401175904E216C4B8F017C4B9F0AC
:1009E00034DF0001010EB26F0401080E016F100E1A
:1009F000026F040E036F800E006F0401180E066F65
:100A0000040E076FC80E046F10D00001020EB26F03
:100A10000401056BC80E046F0401080E016F180E67
:100A2000026F040E036FC80E006F12000001B26B5C
:100A30000401080E016F100E026F040E036F880E82
:080A4000006F0401046B1200B9
:080A4800040110511F0B01080D
:100A500001E079D0145101E076D0060E115D2EE14F
:100A60001351230A28E0010A13E0030A01E024D00D
:100A70000001020EB36F0001BC0505E10001020E8A
:100A8000B46F0E0EB56F090E0001B86FB96B14D0BC
:100A90000001020EB36F0001BC0505E10001E10E8B
:100AA000B46F0E0EB56F0001BC0504E11D0E000110
:100AB000B86FB96B01D000D00001BB8304011051A5
:100AC000600BE842E842E842E842E842010801E0FF
:100AD0003AD011510B0A31E0080A21E0090A19E065
:100AE000080A09E00B0A05E0080A01E02CD02CD81E
:100AF0002AD02BD828D00001020EB36F0001BE0E01
:100B0000B46F000EB56F0001BB930001010EB86F0A
:100B10001AD00001020EB36F13C4BEF014D000014E
:100B2000020EB36F0001BF0EB46F000EB56F00016F
:100B3000BB930001010EB86F06D00001020EB36F27
:100B400012C4BFF000D01200120012000001C06BEE
:100B50001E0E716E0401400E096F200E0A6F040E06
:100B60000B6F880E086F0401600E0E6F040E0F6F7E
:100B7000400E0C6F1200D9CFE6FFE1CFD9FFE6524D
:100B8000FC0EDB50400805E2400EF36EFC0EF3CF86
:100B9000DBFFDF6AFC0EDB50DF5C19E2DF50E76E43
:100BA000FD0EDBCFE9FFFE0EDBCFEAFFE750E926C3
:100BB000000EEA22EF50E66EDF50EA6A600FE96E3F
:100BC000040EEA22E552E750EF6EDF2AE3D7FC0E6F
:100BD000DBCF0DF4400E04010C170C7D880E0C13B6
:100BE000E552E552E7CFD9FF1200D9CFE6FFE1CFBA
:100BF000D9FF0001C06B040108BF30D0FC0EDBCF71
:100C000000F00951D880005403E2FC0E09C4DBFF58
:100C10000001C06BFC0EDB50C05D19E2C051EA6AF6
:100C2000200FE96E040EEA22EF50E66EC051E76E27
:100C3000FD0EDBCFE9FFFE0EDBCFEAFFE750E92632
:100C4000000EEA22E552E750EF6EC02BE3D7040115
:100C5000400E096F0817087D880E08130001C05167
:0A0C600000D0E552E7CFD9FF1200E3
:060C6A006DA60FD802D0B8
:100C70006DB613D80001BA0508E16DBA06D0686AEE
:100C8000696A69806988020EBA6F12006D6A696AC2
:100C90006D860001010EBA6F12006D6A696A00016B
:100CA000BA6B12004DEF06F00001BA5101E13AD0E3
:100CB0006850040B04E06950040B01E038D86DB2B1
:100CC00031D06850010B04E06950010B01E050D8AD
:100CD0006850100B04E06950100B01E024D86850F4
:100CE000400B04E06950400B01E037D86850200BFE
:100CF00004E06950200B01E032D86850020B04E098
:100D00006950020B01E032D8030E0001BA5D01E226
:100D100009D06850080B06E06950080B03E0B0ECFE
:100D200003F068961200698468986D8212006D92D3
:100D30006994689412000001BBA10ED0F8DF6D84A5
:100D40000001080EC16F070EC26FC107000EC25B23
:100D5000C151C211FAE16D941200689C120070A09A
:100D600003D016EC05F07090689A12006892120099
:100D70006A6A686A9F0E6B6E7B0E696E6E6A0F0EF2
:100D8000E66E710EE66E0F0EE66E14D8E552E55271
:100D9000E552160E706E68A602D06896FCD76D9864
:100DA00016EC05F00001BB910001BC6B0001030EC5
:100DB000BA6F1200D9CFE6FFE1CFD9FFFD0EDBCF2E
:100DC000E9FFFE0EDBCFEAFFFC0EDB5004E0EE6A2B
:0E0DD000FC0EDB06F9D7E552E7CFD9FF120083
:020DDE00120100
:100DE0000002000000088117F2080100010203025E
:100DF00009022900010102803209040000020300F7
:100E00000000092101000001221D000705810340A7
:100E1000000107050103400001090220000102044E
:100E200080320904000002FF000000070581034032
:100E3000000107050103400001040309042E0377A4
:100E400000770077002E006700610064006700658E
:100E5000007400700061007200610064006900733A
:100E60000065002E0063006F006D003C03470061C9
:100E7000006400670065007400500061007200614A
:100E800000640069007300650020004800490044C8
:100E900000200042006F006F0074006C006F006162
:100EA00000640065007200100348004900440042DD
:100EB000004F004F0054002A0348004900440042FC
:100EC000004F004F005400200043006F006E00668A
:100ED000006700750072006100740069006F006EA9
:100EE000000600FF0901A10119012940150026FF94
:100EF00000750895408102190129409102C0F00D4A
:0E0F0000190E390E3D0E6B0EA70EB70E480AE5
:020F0E00D9CF39
:100F1000E6FFE1CFD9FF030EE1260F0EC16E9386E7
:100F2000580EE66E39EC08F0E55281A60DD0FE0EA3
:100F3000F66E5F0EF76EF86A0800F550DF6E550E1C
:100F4000DF5C02E100EF10F033D83DD893EC01F004
:100F5000D950010FE96EDACFEAFFEE50ED100AE149
:100F6000980EF36E010EF3CFDBFF3A0EF36E020E16
:100F7000F3CFDBFF010EDBCF00F0020EDBCF01F081
:100F80004C0E005C1D0E015802E28B8C01D08B9C34
:100F9000010EDB06020E01E2DB06D7D7030EE15C91
:100FA00002E2E16AE552E16EE552E7CFD9FF1200B5
:100FB000140E6F6E0001BA6B0001BB6B0001BC6BBD
:100FC0008B9C949C120035EC06F06FBE02D054EC62
:040FD00006F0120015
:0C0FD4002A0EF66E000EF76E000EF86E8E
:100FE00000010900F550AD6F0900F550AE6F03E147
:100FF000AD6701D03DD00900F550A86F0900F5504C
:10100000A96F0900F550AA6F09000900F550E96EB3
:101010000900F550EA6E090009000900F550AB6FB0
:101020000900F550AC6F09000900F6CFAFF0F7CF1B
:10103000B0F0F8CFB1F0A8C0F6FFA9C0F7FFAAC082
:10104000F8FF0001AB5302E1AC5307E00900F55093
:10105000EE6EAB07F8E2AC07F9D7AFC0F6FFB0C051
:10106000F7FFB1C0F8FF0001AD07000EAE5BBFD7C0
:0210700012006C
:0E107200FF0EE350076EEF0E01D0F30EE76E97
:10108000E72E40EF08F00C0E066EE76AE72E46EFFB
:1010900008F0062E45EF08F0072E3EEF08F012008C
:1010A00013EE00F023EE00F0F86A059CEAEC07F07E
:0C10B00065EC08F087EC07F0FBD712009D
:0410BC0000EE00F052
:0A10C0000F0EEE6AEA62FDD712007F
:0210CA00120012
:020000040030CA
:0100000028D7
:010001000EF0
:0100020026D7
:010003001EDE
:010005008179
:010006008178
:010008000FE8
:01000900C036
:01000A000FE6
:01000B00E014
:01000C000FE4
:01000D0040B2
:00000001FF
